:100000000C9455020C947D020C947D020C947D029C
:100010000C947D020C947D020C947D020C947D0264
:100020000C947D020C947D020C947D020C947D0254
:100030000C947D020C947D020C947D020C947D0244
:100040000C94522C0C947D020C944F2E0C949D2EEB
:100050000C947D020C947D020C947D020C947D0224
:100060000C947D020C947D0269174317EE18E21779
:10007000CC179B185517EE1885173A174C178A1886
:10008000CF17A417D7185E178017EB18DE1876184D
:100090007F1892188D18EE189A029E02A302A702EA
:1000A000B102B602BD02C202C802CD02D202D7021C
:1000B000DE02E602EE02F402F902FF020B03130372
:1000C00018031F0326032E03485454502F312E309B
:1000D0002034303120556E617574686F72697A65AD
:1000E000640A436F6E74656E742D547970653A209E
:1000F000746578742F68746D6C0A3C68313E3430D6
:100100003120556E617574686F72697A65643C2F31
:1001100068313E0057616B652075700A004D61695A
:100120006E74656E616E63650A004C6E646B20547C
:1001300072616365722076302E38612C2028632925
:100140004C65204E6574206475204B65726D657535
:100150007220323031330A002C2047617465776198
:10016000793A20002C204E65746D61736B3A200043
:10017000495020616464726573733A2000206D56A3
:100180000A00206D562C2056696E3A2000206279B4
:100190007465732C205663633A20004672656520AF
:1001A0006D656D6F72793A20006261636B20746FC8
:1001B000203139322E3136382E312E32350A006454
:1001C0006F6E650A0052657175657374696E67209C
:1001D00049502041646472657373202E2E2E2000D6
:1001E0003C68313E323030204F4B3C2F68313E006E
:1001F0000A3C2F626F64793E0A3C2F68746D6C3E36
:100200000A003C68746D6C3E3C686561643E3C74F9
:1002100069746C653E4C6E646B20547261636572E8
:100220003C2F7469746C653E3C2F686561643E0ABE
:10023000003C626F64793E3C68313E4C6E646B20DA
:100240005472616365722076657273696F6E207691
:10025000302E38613C2F68313E0A00485454502FEC
:10026000312E3020323030204F4B0D0A436F6E74E8
:10027000656E742D547970653A20746578742F68B2
:10028000746D6C0D0A507261676D613A206E6F2D4E
:1002900063616368650D0A0D0A00414343004144F0
:1002A000445200434D440044454C45535441474556
:1002B0000044554D5000454550524F4D0047415464
:1002C0004500484953544F004C4F4144004D414371
:1002D00041004D41534B004D454D4F5259004D4546
:1002E0005355524553004D4F444545434F005041EF
:1002F00052414D00504F5254005245534554005303
:10030000455249414C4445425547005354414E449F
:1003100042590054494D4500555054494D450056E9
:10032000494E4D415800564F4C54414745005741A6
:10033000544348444F4700000108000604000145AB
:1003400000008200004000200D0A436F6E74656E4D
:10035000742D547970653A206170706C69636174B2
:10036000696F6E2F782D7777772D666F726D2D758B
:10037000726C656E636F6465640D0A0D0A00436FED
:100380006E74656E742D4C656E6774683A20000D4E
:100390000A557365722D4167656E743A204574681D
:1003A0006572536869656C642F312E360D0A41639E
:1003B000636570743A202A2F2A0D0A436F6E6E65AA
:1003C0006374696F6E3A20636C6F73650D0A000D7C
:1003D0000A0020485454502F312E310D0A486F73B3
:1003E000743A2000504F5354200020000D0A5573DA
:1003F00065722D4167656E743A2045746865725365
:100400006869656C642F312E360D0A41636365702F
:10041000743A20746578742F68746D6C0D0A436F9C
:100420006E6E656374696F6E3A20636C6F73650DF1
:100430000A0D0A0020485454502F312E310D0A481D
:100440006F73743A200047455420000000000024D8
:100450000027002A0000000000250028002B0000D3
:1004600000000023002600290004040404040404FE
:100470000402020202020203030303030301020453
:100480000810204080010204081020010204081016
:100490002000000007000201000003040600000025
:1004A00000000000000097070B3011241FBECFEFA3
:1004B000D8E0DEBFCDBF15E0A0E0B1E0E6E9F5E6AB
:1004C00002C005900D92AE39B107D9F717E0AEE939
:1004D000B5E001C01D92A63EB107E1F714E0CAEAFB
:1004E000D4E004C02297FE010E948E32C63AD107A2
:1004F000C9F70E9461300C94C9320C940000A0E04E
:10050000B0E0E5E8F2E00C949A32EC01A880B98002
:10051000CA80DB80A114B104C104D10441F484E297
:10052000A82E89EDB82E8BE5C82E87E0D82EC601FF
:10053000B5012DE133EF41E050E00E94713227EA2E
:1005400031E440E050E00E9409327B018C01C60199
:10055000B5012DE133EF41E050E00E947132CA0154
:10056000B9012CEE34EF4FEF5FEF0E9409326E0DB0
:100570007F1D801F911F97FF04C061507040804015
:100580009048688379838A839B839B013F77C90165
:10059000CDB7DEB7EAE00C94B6320E947F02089530
:1005A00084E291E00E947F020895A0E0B0E0809391
:1005B000240190932501A0932601B093270108956B
:1005C000FC0105900020E9F7809590958E0F9F1F04
:1005D0000895FB01DC014150504030F08D910590B1
:1005E000801919F40020B9F7881B990B0895DC01D4
:1005F00001C06D9341505040E0F70895FB01DC01CC
:100600004150504030F08D910190801919F4002034
:10061000B9F7881B990B0895EF92FF920F931F93E0
:10062000CF93DF93EC01A0E0B0E0EE24FF2487013C
:1006300009C0F901EA0FFB1F8081E80EF11C011DC2
:10064000111D1196A617B707A4F3452B69F09B015E
:10065000442737FD4095542FB701C8010E944F32FF
:10066000C901DA017C018D01D801C701807F90703A
:10067000A070B07024E0B695A795979587952A95B8
:10068000D1F78A3010F0895C01C0805DFE01E95825
:10069000FB4F80839E012F5F3F4F6E2D6F706A303E
:1006A00010F0695C01C0605DF901E958FB4F60839F
:1006B0002F5F3F4FF901E958FB4F80E280832F5FA6
:1006C0003F4FC901DF91CF911F910F91FF90EF90A4
:1006D0000895EF92FF920F931F93CF93DF93EC0156
:1006E000FA0120E030E0EE24FF2487010AC0819166
:1006F0009191A0E0B0E0E80EF91E0A1F1B1F2F5FCA
:100700003F4F261737079CF39B01442737FD409541
:10071000542FC801B7010E944F3279018A01D801D4
:10072000C7016CE0B695A795979587956A95D1F71F
:100730008F708A3010F0895C01C0805DFE01E9583D
:10074000FB4F80839E012F5F3F4FBB27A12F902F30
:100750008F2D8F708A3010F0895C01C0805DF901A7
:10076000E958FB4F80832F5F3F4FD801C701807F3F
:100770009070A070B07044E0B695A7959795879556
:100780004A95D1F78A3010F0895C01C0805DF9018B
:10079000E958FB4F80832F5F3F4F4E2D4F704A30FB
:1007A00010F0495C01C0405DF901E958FB4F4083FE
:1007B0002F5F3F4FF901E958FB4F80E280832F5FA5
:1007C0003F4FC901DF91CF911F910F91FF90EF90A3
:1007D00008959C01DB01CA01FCE1B695A7959795A8
:1007E0008795FA95D1F78A30910514F0895C01C09C
:1007F000805DF901E958FB4F80832F5F3F4FDB019C
:10080000CA0180709070A070BF708B2F9927AA27A3
:10081000BB278A30910514F0895C01C0805DF90125
:10082000E958FB4F80832F5F3F4FDB01CA01807087
:100830009070A07FB070F4E1B695A79597958795D5
:10084000FA95D1F78A30910514F0895C01C0805D7A
:10085000F901E958FB4F80832F5F3F4FDB01CA014D
:1008600080709070AF70B070CD01AA27BB278A301E
:10087000910514F0895C01C0805DF901E958FB4FD6
:1008800080832F5F3F4FDB01CA018070907FA07093
:10089000B070FCE0B695A79597958795FA95D1F736
:1008A0008A30910514F0895C01C0805DF901E95836
:1008B000FB4F80832F5F3F4FDB01CA0180709F7029
:1008C000A070B070892F9A2FAB2FBB278A3091056B
:1008D00014F0895C01C0805DF901E958FB4F808309
:1008E0002F5F3F4FDB01CA01807F9070A070B07016
:1008F00074E0B695A795979587957A95D1F78A3044
:10090000910514F0895C01C0805DF901E958FB4F45
:1009100080832F5F3F4F4F7050704A30510514F065
:10092000495C01C0405DF901E958FB4F40832F5FEE
:100930003F4FF901E958FB4F80E280832F5F3F4F23
:10094000C9010895DC01FC01E95AFE4FE0818E2FB8
:1009500080538A3038F08151863010F080E002C038
:100960008E2F8753982F9295907FA95ABE4F11963C
:10097000EC918E2F80538A3010F4892B08958E2F9E
:100980008154863010F080E008958E2F8753892B94
:1009900008950F931F93CF93DF938C01E091A205ED
:1009A000EE2309F400C120919E05222369F4809171
:1009B0009F05882349F48091A005882329F480911C
:1009C000A105882309F4EFC040E0A0E08A2F90E061
:1009D000880F991F50E04E1708F451E0A52FA82B5F
:1009E0004F5F483099F760E0862F90E0880F991F9D
:1009F00050E04E1708F451E0652F682B4F5F4031EF
:100A000099F770E0872F90E0880F991F50E04E17FC
:100A100008F451E0752F782B4F5F483199F780E04B
:100A200090E0880F991F50E04E1708F451E0582BC2
:100A3000852F4F5F4032A1F7F801E95AFE4F8081C0
:100A4000C82FD0E08A2F90E08C239D2330E08217BE
:100A5000930729F5862F90E0218130E082239323AC
:100A600020919F0530E082179307C9F4872F90E00B
:100A7000228130E0822393232091A00530E0821769
:100A8000930769F4852F90E0238130E0822393233C
:100A90002091A10530E08217930709F484C0E0910A
:100AA000A705EE2309F47CC02091A305222369F455
:100AB0008091A405882349F48091A505882329F411
:100AC0008091A605882309F46BC0F72F40E08F2F93
:100AD00090E0880F991F50E04E1708F451E0F52F71
:100AE000F82B4F5F483099F7672F862F90E0880FDB
:100AF000991F50E04E1708F451E0652F682B4F5FA7
:100B0000403199F7872F90E0880F991F50E04E17DA
:100B100008F451E0752F782B4F5F483199F750E07A
:100B2000852F90E0880F991F50E04E1708F451E090
:100B3000A52FA82B5A2F4F5F403291F78F2F90E0AF
:100B40008C239D2330E08217930751F5862F90E088
:100B5000F801E95AFE4F218130E08223932320914E
:100B6000A40530E082179307D9F4872F90E0228103
:100B700030E0822393232091A50530E0821793076C
:100B800079F440E050E08A2F90E0238130E0822326
:100B900093232091A60530E08217930731F403C018
:100BA00040E050E002C041E050E0CA01DF91CF9147
:100BB0001F910F910895FC0150814181A82FFC01E4
:100BC00070E062507040B0E131E416C0228190E0E4
:100BD000852F880F47FD8F5F440F27FD4F5F57FD1F
:100BE00002C0582F03C0582F5B2743279F5F9830C0
:100BF00011F0220FEDCF31968E2F8A1B90E08617D1
:100C0000970724F3952F80E0242F30E0282B392BF1
:100C1000C90108952F923F924F925F926F927F92F7
:100C20008F929F92AF92BF92CF92DF92EF92FF92FC
:100C30000F931F93DF93CF93CDB7DEB728970FB6EF
:100C4000F894DEBF0FBECDBF809117048B3E09F034
:100C500055C180911804803909F050C18091190460
:100C60008B3E09F04BC180911A04803909F046C1CE
:100C700080911B048B3E09F041C180911C04803996
:100C800009F03CC189EF95E09C838B83E1E2F6E0BB
:100C9000FA83E98385E3282E86E0382E09E4602E66
:100CA00006E0702E1DE5812E16E0912EB1E7AB2EE9
:100CB000B6E0BB2EABE7CA2EA6E0DA2EF5E8EF2EA3
:100CC000F6E0FF2E07E116E06FE876E049E956E02E
:100CD00023EA36E08DE096E098878F83ADEAB6E0B0
:100CE000E7EBF6E0FE83ED83E8E04E2E512CEB813E
:100CF000FC8180899189938B828BE981FA8180893B
:100D00009189938B828BF10180899189938B828B5E
:100D1000F30180899189938B828BF4018089918979
:100D2000938B828BF50180858187F6018085818791
:100D3000F70180858187F80180858187FB018085A7
:100D40008187FA0180858187F90180858187EF811C
:100D5000F8858085818718968C91189719968C93C1
:100D60001997ED81FE8180899189938B828B0894FC
:100D7000410851088B819C8102979C838B83E98178
:100D8000FA813297FA83E9838EEF9FEF280E391E9E
:100D9000680E791E880E991E0894A108B10808945F
:100DA000C108D1080894E108F108015010406150D1
:100DB00070404150504021503040EF81F8853197CC
:100DC000F887EF8311978D819E8102979E838D8393
:100DD0009FEF49169FEF590609F089CF90912104A2
:100DE00080E02091200430E0822B932B9093FA0531
:100DF0008093F9059091230480E02091220430E053
:100E0000822B932B909322068093210690912704A6
:100E100080E02091260430E0822B932B90933606BD
:100E2000809335069091290480E02091280430E0D9
:100E3000822B932B90934A068093490690912B0422
:100E400080E020912A0430E0822B932B90935E0661
:100E500080935D0680912C048093710680912D040F
:100E600080937B0680912E048093850680912F04C9
:100E7000809317068091300480938F06809131040F
:100E800080939906809132048093A3068091330465
:100E900080930D06809134048093AD0690913604C2
:100EA00080E02091350430E0822B932B9093B8069C
:100EB0008093B706109138040091390410923904D8
:100EC000109238048DE194E06DE10E94DB051093EF
:100ED00038040093390490933B0480933C04809140
:100EE000E2059091E30501969093E3058093E20576
:100EF0001092A9051092A8051092770428960FB6B3
:100F0000F894DEBF0FBECDBFCF91DF911F910F913F
:100F1000FF90EF90DF90CF90BF90AF909F908F9019
:100F20007F906F905F904F903F902F90089586EE46
:100F300095E00E94952A0895AC0186EE95E067E55C
:100F400071E020EF31E00E94452B0895EF92FF926F
:100F50000F931F93AC0106EE15E097E5E92E91E0A3
:100F6000F92EC801B70122E032E00E94452BAC0106
:100F7000C801B70121E332E00E94452B1F910F9178
:100F8000FF90EF90089586EE95E067E571E040E010
:100F900050E02BE532E00E94452B08958EE48093CB
:100FA0007C0062E070E080E090E00E94A82C8091DC
:100FB0007A00806480937A0080917A0086FDFCCF6D
:100FC0008091780090E0A0E0B0E060917900362F49
:100FD00020E0442737FD4095542F282B392B4A2BEE
:100FE0005B2B60E070E381E190E00E947132CA0106
:100FF000B9010895CF93DF93EC010CC06A3029F456
:1010000080EB97E00E94A23004C080EB97E00E9442
:10101000C92F2196FE016491662381F7DF91CF915C
:101020000895AF92BF92CF92DF92EF92FF920F930B
:101030001F93CF93DF935C014091F5055091F60526
:101040004115510579F0C091F705D091F805FE01E1
:10105000EE0FFF1FE856FF4F659174910E94E90261
:10106000892B19F1CC24DD2447E1E42EF12CE60193
:10107000CE0DDF1DD595C795D093F805C093F70524
:10108000FE01EE0FFF1FE856FF4F05911491C801B6
:101090000E94E002AC019093F6058093F505C5012E
:1010A000B8010E94E902009719F4FE01B09611C040
:1010B000181619062CF46E010894C11CD11C04C02A
:1010C0007E010894E108F108EC14FD0484F6E0E0E8
:1010D000F0E0CF01DF91CF911F910F91FF90EF9042
:1010E000DF90CF90BF90AF900895CF92DF92EF92B4
:1010F000FF920F931F93CF93DF93C0905501D09031
:1011000056010E94A42B029709F0E2C00E949A2C7B
:101110002091DA053091DB054091DC055091DD0529
:10112000621B730B840B950B615A7B4B8D40904077
:1011300008F4CEC0809155019091560118161906F9
:101140000CF0C6C08091E2059091E30509970CF47C
:10115000BFC00E949A2C6093DA057093DB058093E0
:10116000DC059093DD05C091E205D091E305CB301D
:10117000D10514F0CAE0D0E0E9EFF5E060E070E0FE
:1011800020E030E040E050E00AC081919191A0E081
:10119000B0E0280F391F4A1F5B1F6F5F7F4F6C172E
:1011A0007D079CF3CA01B9012AE030E040E050E03D
:1011B0000E9409329E01442737FD4095542F0E941A
:1011C0004F3279018A0120E030E040E050E008C071
:1011D000F901E35FF94F8081480F511D2F5F3F4FA9
:1011E0002C173D07ACF320E030E060E070E008C071
:1011F000F901E95EF94F8081680F711D2F5F3F4F44
:101200002C173D07ACF38091450190914601A0E079
:10121000B0E0E816F9060A071B07A8F04C175D07AF
:1012200091F48091490190914A019C01429FC00133
:10123000439F900D529F900D11246817790718F065
:10124000A1E0CA2ED12C8091470190914801A0E0E5
:10125000B0E0E816F9060A071B0788F0452B79F07D
:1012600080914B0190914C019C01C29FC001C39F92
:10127000900DD29F900D11246817790748F5809141
:10128000550190915601019719F51092D6051092CB
:10129000D7051092D8051092D9051092D205109258
:1012A000D3051092D4051092D5051092CE05109258
:1012B000CF051092D0051092D1051092CA05109258
:1012C000CB051092CC051092CD05F2E0CF2ED12C9B
:1012D0008091550190915601039709F062C0809169
:1012E000C6059091C705A091C805B091C905805C5D
:1012F000944DA140B04008F454C00E949A2C209113
:10130000BE053091BF054091C0055091C105621BDB
:10131000730B840B950B2091C6053091C705409146
:10132000C8055091C905220F331F441F551F2617AA
:10133000370748075907A8F51092D6051092D70528
:101340001092D8051092D9051092D2051092D305AB
:101350001092D4051092D5051092CE051092CF05AB
:101360001092D0051092D1051092CA051092CB05AB
:101370001092CC051092CD0586EE95E00E94992A38
:101380000E949A2C6093C2057093C3058093C40594
:101390009093C5051092DF051092DE0572E0C72E0E
:1013A000D12CC601DF91CF911F910F91FF90EF904B
:1013B000DF90CF9008950E94C3070E94A607AC015A
:1013C00086EE95E067E571E027E734E00E943F2B69
:1013D0000E949C0708950F931F93CF93DF938C0176
:1013E0000E94DF2B0E94A42B805D80937704809164
:1013F000E2059091E305409734F08FE090E0909300
:10140000E3058093E2058091E2059091E3058A303F
:10141000910514F0895C01C0805D8093780480910F
:101420005501805D809379048091DE05805D809315
:101430007A0480E280937B040E94DF2BAB01BC0125
:1014400085E090E00E94E903FC011016110634F5D6
:10145000C7E1D4E0DC01A958BB4F20E29881892F75
:1014600082958F708A3010F0895C01C0805D8C930A
:10147000892F8F708A3010F0895C01C0805D1196D1
:101480008C93119712962C9312972196139684E0C1
:10149000CF33D80719F7E858FF4F6DC06091E205C8
:1014A0007091E305161617060CF065C0EB016B3062
:1014B000710514F0CAE0D0E0CF01BE0149EF55E05C
:1014C0000E946903BE0141E256E00E946903BE0129
:1014D00045E356E00E946903BE0149E456E00E94DC
:1014E0006903BE014DE556E00E946903BE0147EB6A
:1014F00056E00E946903BE0140E050E021E736E07B
:101500000E940C03BE0140E050E02BE736E00E9451
:101510000C03BE0140E050E025E836E00E940C03D9
:10152000BE0141E050E027E136E00E940C03BE011D
:1015300040E050E02FE836E00E940C03BE0140E09E
:1015400050E029E936E00E940C03BE0140E050E083
:1015500023EA36E00E940C03BE0140E050E02DE09B
:1015600036E00E940C03BE0141E050E02DEA36E077
:101570000E940C03FC01F093AB05E093AA05E95827
:10158000FB4F108287E591E00E94DB09012B21F4DB
:101590001092E3051092E205DF91CF911F910F9118
:1015A00008955F926F927F928F929F92AF92BF92B7
:1015B000CF92DF92EF92FF920F931F93CF93DF931F
:1015C0003C010E94DF2B0E94A42B805D8093770456
:1015D0008091E2059091E305409734F08FE090E030
:1015E0009093E3058093E2058091E2059091E305F5
:1015F0008A30910514F0895C01C0805D8093780485
:1016000080915501805D809379048091DE05805D35
:1016100080937A0480E280937B040E94DF2BAB01ED
:10162000BC0185E090E00E94E903EC0185E10E94A5
:10163000462DAA24BB24812C14E0912E00E010E05A
:10164000CC24DD247601B0E25B2E64E170E080E022
:1016500090E00E94A82C85E10E94462D9C018815EF
:1016600099050CF44C01021713070CF4890161145D
:10167000710429F084E0A816B10409F047C0E3E042
:10168000293E3E0764F0FE01E958FB4FC90168EEB0
:1016900073E00E943C32605D6083219603C0253672
:1016A000310584F0FE01E958FB4FC90168EE73E093
:1016B0000E943C3264E670E00E943C32605D6083D0
:1016C000219603C02B3031057CF0FE01E958FB4F19
:1016D000C90164E670E00E943C326AE070E00E945A
:1016E0003C32605D60832196FE01E958FB4FC901E1
:1016F0006AE070E00E943C32805D8083CE010196FA
:10170000FC01E958FB4F5082EC012196C901AA2740
:1017100097FDA095BA2FC80ED91EEA1EFB1E08948D
:10172000A11CB11CF7E0AF16B10409F08ECF080D73
:10173000191DC801AA2797FDA095BA2FC81AD90A62
:10174000EA0AFB0AA0904301B0904401950140E0F1
:1017500050E0C701B6010E94093220E034E140E0C8
:1017600050E00E944F3269017A01FE01E958FB4FB7
:1017700088E28083219681E1C81687E2D80680E05E
:10178000E80680E0F80680F08E0109581B4FC7017B
:10179000B60120E137E240E050E00E944F32205D88
:1017A000F8012083219609C0F9EECF16F3E0DF0699
:1017B000F0E0EF06F0E0FF06B0F08E0109581B4F95
:1017C000C701B60120E137E240E050E00E944F320D
:1017D00028EE33E040E050E00E944F32205DF801F7
:1017E0002083219606C0F5E6CF16D104E104F1046A
:1017F000B0F08E0109581B4FC701B60128EE33E047
:1018000040E050E00E944F3224E630E040E050E0FB
:101810000E944F32205DF8012083219606C0FBE034
:10182000CF16D104E104F104A8F08E0109581B4F32
:10183000C701B60124E630E040E050E00E944F329C
:101840002AE030E040E050E00E944F32205DF80195
:10185000208321968E0109581B4FC701B6012AE04B
:1018600030E040E050E00E944F32605DF80160835C
:10187000CE010196FC01E958FB4F30E2308301961E
:10188000FC01E958FB4F2DE620830196FC01E95845
:10189000FB4F26E520830196FC01E958FB4F29E226
:1018A0002083DC011196672809F47DC0FD01E95809
:1018B000FB4F3083CD010196FC01E958FB4F2DE42D
:1018C00020830196FC01E958FB4F21E62083019615
:1018D000FC01E958FB4F28E720830196FC01E958F9
:1018E000FB4F2AE320839C012F5F3F4FF1E1AF16AE
:1018F000F7E2BF0668F0F901E958FB4FC50160E166
:1019000077E20E942832605D60832F5F3F4F05C001
:1019100089EEA81683E0B80688F0F901E958FB4F74
:10192000C50160E177E20E94283268EE73E00E9410
:101930002832605D60832F5F3F4F04C0E5E6AE163E
:10194000B10488F0F901E958FB4FC50168EE73E076
:101950000E94283264E670E00E942832605D608355
:101960002F5F3F4F04C0FBE0AF16B10480F0F901D8
:10197000E958FB4FC50164E670E00E9428326AE036
:1019800070E00E942832605D60832F5F3F4FF90155
:10199000E958FB4FC5016AE070E00E942832805D83
:1019A0008083D9011196A958BB4F1C9287E591E01D
:1019B0000E94DB09DF91CF911F910F91FF90EF9073
:1019C000DF90CF90BF90AF909F908F907F906F905F
:1019D0005F9008950F931F93DF93CF9300D0CDB7FF
:1019E000DEB70E94A42B805D809377048091E2058E
:1019F0009091E305409734F08FE090E09093E305F9
:101A00008093E2058091E2059091E3058A3091058B
:101A100014F0895C01C0805D809378048091550149
:101A2000805D809379048091DE05805D80937A04E7
:101A300010E210937B040E94DF2BAB01BC0185E018
:101A400090E00E94E903FC01E958FB4F26E4208363
:101A50000196FC01E958FB4F22E720830196FC0127
:101A6000E958FB4F25E620830196FC01E958FB4F1E
:101A700020830196FC01E958FB4F2AE3208301965D
:101A8000FC01E958FB4F10838C010F5F1F4F8091C1
:101A9000E2079091E307009711F486EE97E09E012C
:101AA0002F5F3F4F281B390B87E22031380718F092
:101AB00020E030E038C083E0293E38076CF0F801C0
:101AC000E958FB4FC90168EE73E00E943C32605D4B
:101AD00060830F5F1F4F03C0253631058CF0F8017E
:101AE000E958FB4FC90168EE73E00E943C3264E69E
:101AF00070E00E943C32605D60830F5F1F4F03C047
:101B00002B30310584F0F801E958FB4FC90164E638
:101B100070E00E943C326AE070E00E943C32605DFE
:101B200060830F5F1F4FF801E958FB4FC9016AE05E
:101B300070E00E943C32805D8083F8013196DF01C5
:101B4000A958BB4F80E28C933196DF01A958BB4F57
:101B500082E68C933196DF01A958BB4F89E78C93BD
:101B60003196DF01A958BB4F84E78C933196DF0192
:101B7000A958BB4F85E68C93E858FB4F83E78083D9
:101B8000118287E591E00E94DB090F900F90CF91C1
:101B9000DF911F910F9108950F931F930E94A42B23
:101BA000805D809377048091E2059091E3054097F2
:101BB00034F08FE090E09093E3058093E20580910C
:101BC000E2059091E3058A30910514F0895C01C02B
:101BD000805D8093780480915501805D80937904C5
:101BE0008091DE05805D80937A0480E280937B049F
:101BF0000E94DF2BAB01BC0185E090E00E94E9036D
:101C00008C010E94DF2BAB01BC018091AE0590914D
:101C1000AF05A091B005B091B105481B590B6A0BF7
:101C20007B0BC8010E94E903FC019093AB058093F4
:101C3000AA05E958FB4F108287E591E00E94DB0975
:101C40001F910F9108957F928F929F92AF92BF92B2
:101C5000CF92DF92EF92FF920F931F93CF93DF9378
:101C6000EC01672B09F4A8C080E091E0BE0144E0DC
:101C700050E00E94FE02009709F09EC0FC8005E043
:101C800010E0AA24BB2465011DC0C601B5012AE0ED
:101C900030E040E050E00E9409322F2D332727FD2D
:101CA0003095205330405901CC24B7FCC094DC2C33
:101CB000A60EB71EC81ED91EFE01E00FF11FF08050
:101CC0000F5F1F4F8F2D80538A3018F40F3011058E
:101CD000E1F6B801615070406C0F7D1F85E091E026
:101CE00044E050E00E94FE02009709F047C0FE0168
:101CF000E00FF11F738084E0882E912C800E911EDE
:101D0000EF01EE24FF2487011BC0C801B7012AE0C0
:101D100030E040E050E00E940932272D332727FDB4
:101D200030952053304079010027F7FC0095102FA3
:101D3000E60EF71E081F191F7B800894811C911C5A
:101D4000872D80538A3028F4219669E18616910404
:101D5000E4F2A8019701D801C70188579040A0403C
:101D6000B040895A9B41A040B04020F020EB34E0C5
:101D700040E050E0CA01B9010E94A92B0E94A42BA7
:101D8000892BB1F40E949A2C28EE33E040E050E019
:101D90000E944F32D601C501821B930BA40BB50BD9
:101DA0008093AE059093AF05A093B005B093B105B5
:101DB000C601B5010E94B22B0E94CC0DDF91CF91DC
:101DC0001F910F91FF90EF90DF90CF90BF90AF9059
:101DD0009F908F907F900895CF92DF92EF92FF9225
:101DE0000F931F93CF93DF9391E0909377048093A9
:101DF000780460937904ABECB6E0CAE7D4E0E62F50
:101E0000F0E09F012A0F3B1F02C08D918993A2171A
:101E1000B307D9F72AE7E22E24E0F22EEE0EFF1EDA
:101E2000D7011C928F0105581B4FD8011C9295E0D9
:101E3000C92ED12CCE0EDF1EF601E958FB4F8FE7DD
:101E400080836B5F87E794E00E94DB05F701908356
:101E5000D8018C93C0E0D0E08091E4059091E50535
:101E6000892B59F080EB97E06BEE0E94C92F80EB35
:101E700097E060E90E94C92F1AC080EB97E06BEEF3
:101E800070E040E150E00E94A33180EB97E060E217
:101E90000E949A3080EB97E060E970E040E150E00A
:101EA0000E94A33180EB97E060E20E949A30219675
:101EB000C330D10589F6C7E7D4E000E010E0809197
:101EC000E4059091E505892B21F080EB97E068818E
:101ED0000AC080EB97E0688140E150E00E945131F8
:101EE00080EB97E060E20E94C92F0F5F1F4F2196A1
:101EF000C016D10624F78091E4059091E505892B61
:101F000021F480EB97E00E94A230DF91CF911F91E6
:101F10000F91FF90EF90DF90CF9008951092CB0635
:101F2000892B19F081E08093CB061092CC068AEAC7
:101F300061E00E94EC0E0895CF93DF93C0E0D0E003
:101F40008EE097E0BE010E94912BFE01E95EFB4FFF
:101F500080832196C034D10599F71092570480915F
:101F600017048D34A9F580911804813489F55091B6
:101F7000190440911A0430911B0420911C04909183
:101F80001D0480911E04552359F44423A9F43323DE
:101F900099F4222389F4992379F4882369F418C0E9
:101FA0005F3F51F44F3F41F43F3F31F42F3F21F465
:101FB0009F3F11F48F3F61F0509328014093290116
:101FC00030932A0120932B0190932C0180932D01B3
:101FD00080911F04813421F580912004843401F51F
:101FE000809121048434E1F4809122048235C1F48B
:101FF000309123042091240490912504809126049B
:102000003F3F31F42F3F21F49F3F11F48F3F41F0C8
:1020100030932E0120932F01909330018093310152
:1020200080912F04873469F580913004813449F51B
:1020300080913104843529F580913204853409F585
:10204000309133042091340490913504809136040A
:10205000332339F4222369F4992359F4882349F46A
:1020600010C03F3F31F42F3F21F49F3F11F48F3FC9
:1020700041F03093320120933301909334018093E7
:102080003501809137048035B1F4809138048F3464
:1020900091F480913904823571F480913A04843549
:1020A00051F480913B0490913C04882311F49923CE
:1020B00011F09093420180913D04813409F073C086
:1020C00080913E04833409F06EC080913F048334D4
:1020D00009F069C080914004813309F064C04091E7
:1020E0004104309142042091430490914404509162
:1020F0004504852F8150803208F055C0442339F4BF
:10210000332371F4222361F4992351F44CC04F3FDF
:1021100039F43F3F29F42F3F19F49F3F09F443C09E
:1021200040939E0530939F052093A0059093A105B1
:102130005093A205809146048134A9F5809147040B
:10214000833489F580914804833469F5809149048A
:10215000823349F540914A0430914B0420914C045C
:1021600090914D0450914E04852F81508032D8F4C7
:10217000442339F4332369F4222359F4992349F48D
:1021800012C04F3F31F43F3F21F42F3F11F49F3FE6
:1021900051F04093A3053093A4052093A505909397
:1021A000A6055093A70580914F048234E1F48091F5
:1021B00050048635C1F4809151048934A1F4809192
:1021C00052048E3481F4209153043091540422231C
:1021D00011F4332341F0922F80E0830F911D9093EF
:1021E00044018093430180915B048335E1F4809145
:1021F0005C048435C1F480915D048234A1F4809143
:102200005E048C3481F420915F04309160042223B9
:1022100011F4332341F0922F80E0830F911D9093AE
:10222000480180934701809161048335E1F48091F6
:1022300062048F34C1F4809163048334A1F48091EB
:102240006404883481F4209165043091660422236B
:1022500011F4332341F0922F80E0830F911D90936E
:102260004A0180934901809167048335E1F48091AC
:1022700068048F34C1F4809169048334A1F480919F
:102280006A048C3481F420916B0430916C04222315
:1022900011F4332341F0922F80E0830F911D90932E
:1022A0004C0180934B01DF91CF9108955F926F9223
:1022B0007F928F929F92AF92BF92CF92DF92EF92D6
:1022C000FF920F931F93CF93DF937C010E94C3076C
:1022D0000E94A6076C01F694FE2CEE24F794E79476
:1022E0008F2D8F708A3010F0895C01C0805D8093E3
:1022F0007704C701B4E096958795BA95E1F78870A1
:10230000805D8093780480E3809379048AE38093EE
:102310007A0480E280937B048701C5E0D0E0A0E8E6
:10232000AA2EB12CAE0CBF1CFDE05F2EEAE06E2E93
:1023300070E3772E6AE3862E50E2952E84C0E01675
:10234000F1060CF057C0C8018F709070892B09F00E
:1023500051C0FE01E958FB4F5082CE010196FC01AD
:10236000E958FB4F60829C012F5F3F4F812F8F7098
:102370008A3010F0895C01C0805DF901E958FB4F9B
:1023800080832F5F3F4FC801807F907044E0959518
:1023900087954A95E1F78A3010F0895C01C0805D2D
:1023A000F901E958FB4F8083C9010196FC01E95806
:1023B000FB4F70820196FC01E958FB4F8082019629
:1023C000FC01E958FB4F9082EC012196C8018F7304
:1023D0009070892B79F4C958DB4F188286EE95E00E
:1023E00067E571E0A60127E734E00E943F2B6C010E
:1023F000C0E0D0E08EE097E0B8010E94912B982FCA
:1024000092959F70282F2F709A3018F0892F895C31
:1024100002C0892F805DFE01E958FB4F8083CE0109
:1024200001962A3010F0295C01C0205DFC01E958BA
:10243000FB4F20830196FC01E958FB4F9082EC0191
:1024400021960F5F1F4F0A151B0509F078CFC95859
:10245000DB4F188286EE95E067E571E0A60127E77D
:1024600034E00E943F2B0E949C07DF91CF911F9187
:102470000F91FF90EF90DF90CF90BF90AF909F9023
:102480008F907F906F905F900895CF92DF92EF9240
:10249000FF920F931F93CF93DF938C017B01EA018F
:1024A00069018EE097E06EE370E043E50E94982BAF
:1024B0008EE097E06FE370E044E50E94982B8EE099
:1024C00097E060E470E042E40E94982B8EE097E091
:1024D00061E470E048E40E94982B8EE097E062E4AB
:1024E00070E0412F0E94982B8EE097E063E470E04B
:1024F000402F0E94982B8EE097E064E470E043E563
:102500000E94982B8EE097E065E470E044E50E941D
:10251000982B8EE097E066E470E042E40E94982BEE
:102520008EE097E067E470E04CE40E94982B8EE028
:1025300097E068E470E04F2D0E94982B8EE097E0C2
:1025400069E470E04E2D0E94982B209709F45FC03B
:102550001C141D040CF05BC0CC16DD0608F057C03F
:102560008EE097E06AE470E043E50E94982B8EE0ED
:1025700097E06BE470E04FE40E94982B8EE097E0C8
:102580006CE470E043E40E94982B8EE097E06DE4E9
:1025900070E048E40E94982B8EE097E06EE470E0D3
:1025A0004D2F0E94982B8EE097E06FE470E04C2F47
:1025B0000E94982B8EE097E060E570E043E50E9472
:1025C000982B8EE097E061E570E04FE40E94982B35
:1025D0008EE097E062E570E043E40E94982B8EE085
:1025E00097E063E570E04CE40E94982B4D2D552751
:1025F00047FD5A958EE097E064E570E00E94982BC5
:102600008EE097E065E570E04C2D0E94982BDF91FD
:10261000CF911F910F91FF90EF90DF90CF90089591
:102620004F925F926F927F928F929F92AF92BF92E2
:10263000CF92DF92EF92FF920F931F93CF93DF938E
:102640003C0180E091E0B30144E050E00E94FE02D2
:10265000009709F02FC1F3011481C5E0D0E0882470
:10266000992454011CC0C501B4012AE030E040E0C7
:1026700050E00E940932212F332727FD3095205347
:1026800030404901AA2497FCA094BA2C860E971ECC
:10269000A81EB91EF301EC0FFD1F10812196812F9A
:1026A00080538A3018F4CA30D105E9F6BE01615072
:1026B0007040660D771D85E091E044E050E00E9497
:1026C000FE02009709F0F6C0F301EC0FFD1F5380E6
:1026D0008E010C5F1F4FEF01CC24DD2476011AC060
:1026E000C701B6012AE030E040E050E00E94093224
:1026F000252D332727FD3095205330406901EE24E6
:10270000D7FCE094FE2CC60ED71EE81EF91E5B8097
:102710000F5F1F4F852D80538A3020F4219605319D
:102720001105F4F2B80161507040660D771D8AE022
:1027300091E044E050E00E94FE02009709F07DC065
:10274000A8014A5F5F4FF301E00FF11F2381E80109
:102750002496F301E00FF11F00E010E014C0C8015F
:10276000B3E0880F991FBA95E1F7000F111F080F0A
:10277000191F822F992787FD9095080F191F005365
:10278000104023812196822F80538A3020F4319685
:102790004C175D0724F72801BE0161507040660D9B
:1027A000771D8FE091E044E050E00E94FE02009728
:1027B00019F020E030E02CC0DE011696F301EC0F9A
:1027C000FD1F6381AE014C5F5F4FF301EC0FFD1FF6
:1027D00020E030E015C0C90173E0880F991F7A9599
:1027E000E1F7220F331F280F391F862F992787FD06
:1027F0009095280F391F2053304063814F5F5F4F02
:10280000862F80538A3020F43196A417B5071CF721
:102810000436110594F4201731077CF403331105B5
:1028200064F0293231054CF010934A0100934901BC
:1028300030934C0120934B0104C04424552420E0E4
:1028400030E0C814D904EA04FB04A0F5F8E38F16BD
:10285000F1E39F06F0E0AF06F0E0BF0658F181E437
:1028600088168AE6980680E0A80680E0B80610F58B
:10287000E0E7CE16E0E3DE06E0E0EE06E0E0FE068E
:10288000C8F0F1E9CF16F5E6DF06F0E0EF06F0E07C
:10289000FF0680F49092460180924501D092480153
:1028A000C0924701C401B601A2010E944512C1E0D5
:1028B000D0E002C0C0E0D0E00E94C3070E94A6079B
:1028C000AC01CD2B49F08FE4809377048BE68093A5
:1028D0007804E2E0F0E00AC085E48093770482E7C0
:1028E0008093780480937904E3E0F0E0E958FB4FAB
:1028F0008AE08083118286EE95E067E571E027E744
:1029000034E00E943F2B0E949C07DF91CF911F91E2
:102910000F91FF90EF90DF90CF90BF90AF909F907E
:102920008F907F906F905F904F900895EF92FF92FD
:102930000F931F937C010EE017E0C80168E370E07D
:1029400042E40E94982BC80169E370E046E50E94CA
:10295000982BC8016AE370E049E40E94982BC801F3
:102960006BE370E04EE40E94982B4F2D552747FDF6
:102970005A95C8016CE370E00E94982BC8016DE382
:1029800070E04E2D0E94982B1F910F91FF90EF90B9
:102990000895BF92CF92DF92EF92FF920F931F9311
:1029A000CF93DF936C0180E091E0B60144E050E00A
:1029B0000E94FE02009709F049C0F601B480C5E00C
:1029C000D0E0EE24FF2487011CC0C801B7012AE033
:1029D00030E040E050E00E9409322B2D332727FDE4
:1029E00030952053304079010027F7FC0095102FD7
:1029F000E60EF71E081F191FF601EC0FFD1FB08031
:102A000021968B2D80538A3018F4CA30D105E9F60F
:102A1000D801C701815A9F40A040B04080569D46D2
:102A2000A040B04098F4F0924401E0924301219715
:102A3000CC0DDD1D84E191E0BE0145E050E00E9437
:102A4000FE02009719F4C7010E94961481E090E0FD
:102A50000E94D10ADF91CF911F910F91FF90EF90CB
:102A6000DF90CF90BF9008956F927F928F929F9248
:102A7000AF92BF92CF92DF92EF92FF920F931F938C
:102A8000CF93DF936C018B01695A7E4F80E091E018
:102A900044E050E00E94FE02009719F0C0E0D0E050
:102AA00073C1C80104960E94A204782EE8012696FC
:102AB000CE010E94A204682E80E2C816D10409F457
:102AC00073C1C80108960E94A204882EE8012A96C4
:102AD000CE010E94A204982EC114D10441F086E2D6
:102AE000C816D10421F08FE2C816D10471F42296E1
:102AF000CE010E94A204A82EC114D10439F422965A
:102B0000CE010E94A204B82E07C0AA2488E0C816ED
:102B1000D10409F446C0BB24772059F4662049F457
:102B2000882039F4992029F4AA2019F4BB2009F44B
:102B30002BC188E1C816D10409F472C089E1C81616
:102B4000D1046CF488E0C816D10461F180E1C816A4
:102B5000D10409F446C0C114D10491F00FC086E23B
:102B6000C816D10409F49AC08FE2C816D10409F43A
:102B700095C080E2C816D10409F471C0E601BEC058
:102B80008EE097E060E070E04DE40E94982B8EE0CC
:102B900097E061E070E041E40E94982BC2E0D0E051
:102BA000ADC0BB248EE097E068E070E041E40E9495
:102BB000982B8EE097E069E070E044E40E94982B47
:102BC0008EE097E06AE070E044E40E94982B8EE08B
:102BD00097E06BE070E042E50E94982BCCE0D0E0FB
:102BE0008DC08EE097E060E170E04DE40E94982B8C
:102BF0008EE097E061E170E041E40E94982B8EE066
:102C000097E062E170E043E50E94982B8EE097E048
:102C100063E170E04BE40E94982BC4E1D0E06EC009
:102C20008EE097E068E170E047E40E94982B8EE028
:102C300097E069E170E041E40E94982B8EE097E014
:102C40006AE170E044E50E94982B8EE097E06BE12A
:102C500070E045E40E94982BCCE1D0E04FC08EE0BC
:102C600097E060E270E040E50E94982B8EE097E0EC
:102C700061E270E04FE40E94982B8EE097E062E200
:102C800070E042E50E94982B8EE097E063E270E0EE
:102C900044E50E94982BC4E2D0E030C086010F5F6B
:102CA0001F4F8EE097E0B60141E40E94982B780117
:102CB0000894E11CF11C8EE097E0B80143E40E9407
:102CC000982B87010F5F1F4F8EE097E0B70143E419
:102CD0000E94982BB8016F5F7F4F86E2C816D1041F
:102CE00031F4EB018EE097E0B80141E305C0EB0160
:102CF0008EE097E0B80142E30E94982B8E010F5FAF
:102D00001F4F8EE097E0BE01472D0E94982BE801EF
:102D100021968EE097E0B801462D0E94982B80E224
:102D2000C816D10489F18E010F5F1F4F8EE097E026
:102D3000BE01482D0E94982BE80121968EE097E075
:102D4000B801492D0E94982BC114D10441F086E2AC
:102D5000C816D10421F08FE2C816D104A9F48E015F
:102D60000F5F1F4F8EE097E0BE014A2D0E94982B07
:102D7000CD2811F0E80108C0E80121968EE097E027
:102D8000B8014B2D0E94982BCE01DF91CF911F915E
:102D90000F91FF90EF90DF90CF90BF90AF909F90FA
:102DA0008F907F906F90089588249924AA24B3CEA1
:102DB000AF92BF92DF92EF92FF920F931F93CF9348
:102DC000DF93C091E705D091E805BE01695A7E4FB7
:102DD000FB019E01AE01405C5F4F0AC09081892FCC
:102DE00081568A3110F4905290832F5F3F4F319675
:102DF0002417350720F482E0213C380778F38AE174
:102E000091E044E050E00E94FE02009781F00E94B1
:102E1000C307AC019093E8058093E70586EE95E043
:102E200067E571E020EE31E00E94452BCFC1BE0185
:102E3000655A7E4F8FE191E042E050E00E94FE0231
:102E4000009729F487E591E00E94DB09BFC1CE011C
:102E5000845A9E4F0E941108FC01B097E831F10599
:102E600008F0B9C1EC5CFF4FEE0FFF1F0590F49125
:102E7000E02D09946091E7057091E805675F7F4F49
:102E800080E090E023C06091E7057091E805675FFE
:102E90007F4F88E090E01AC06091E7057091E805E7
:102EA000675F7F4F80E190E011C06091E70570910E
:102EB000E805675F7F4F88E190E008C06091E70513
:102EC0007091E805675F7F4F80E290E00E943415C3
:102ED00085C16091E7057091E805FB01E95AFE4F55
:102EE0008085813329F4675F7F4F86E290E0EECFE3
:102EF000823309F073C1675F7F4F8FE290E0E6CFC6
:102F00001092E1051092E00569C1C091E705D091EA
:102F1000E805BE01605A7E4F80E091E044E050E059
:102F20000E94FE02009709F056C1C95ADE4F6D8516
:102F3000603319F480E090E004C0613341F581E032
:102F400090E00E948E0F23C0C091E705D091E80564
:102F5000BE016D597E4F80E091E044E050E00E9458
:102F6000FE020097A1F4C95ADE4F6889603329F444
:102F700010925601109255010AC0613311F062336C
:102F800031F482E090E0909356018093550181E006
:102F900090E00E94EB091AC181E090E002C080E05D
:102FA00090E00E94EB099093E8058093E7050E946A
:102FB0009A2C6093BA057093BB058093BC059093DF
:102FC000BD058BC084E190E0A0E0B0E08093B60541
:102FD0009093B705A093B805B093B905C091E705E4
:102FE000D091E805BE016B597E4F80E091E044E04E
:102FF00050E00E94FE02009709F067C01092B605EB
:103000001092B7051092B8051092B905FE01E95A61
:10301000FE4FD288C3E1D0E0EE24FF2487015F0198
:103020001FC0C801B7012AE030E040E050E00E9434
:1030300009322D2D30E02053304079010027F7FC74
:103040000095102FE60EF71E081F191FC731D10576
:1030500011F4DD2405C0F501EC0FFD1FD080219691
:103060008D2D80538A3018F4C831D105D0F2E0920A
:10307000B605F092B7050093B8051093B905809195
:10308000B6059091B705A091B805B091B9054E97D6
:10309000A109B10983569145A140B040B0F40E9406
:1030A000DF2B2091B6053091B7054091B8055091BE
:1030B000B905260F371F481F591F2093B2053093BB
:1030C000B3054093B4055093B50582E090E090932A
:1030D000DF058093DE050E949A2C6093B6057093FD
:1030E000B7058093B8059093B90578C08091E7053E
:1030F0009091E805805A9E4F61E070E008C0809191
:10310000E7059091E805805A9E4F60E070E00E94CC
:10311000230E5CC00E94EA0C59C080E090E00E943F
:10312000D10A54C08091E7059091E8058E599E4FD1
:103130000E94C9144BC0C091E705D091E805BE01BB
:103140006E597E4F80E091E044E050E00E94FE0224
:10315000009739F5FE01E95AFE4F6785FE01E959EE
:10316000FE4F40E150E020E030E011C0C901A3E093
:10317000880F991FAA95E1F7220F331F280F391FD7
:10318000260F311D2053304061914F5F5F4F862FD6
:1031900080538A3018F44231510541F7203131050E
:1031A00010F020E030E0C9010E9456110FC086E007
:1031B00090E09093DF058093DE050DC08091E705D8
:1031C0009091E8058D599E4F0E9410139093E80549
:1031D0008093E70503C020E030E002C021E030E04A
:1031E000C901DF91CF911F910F91FF90EF90DF9078
:1031F000BF90AF9008952F923F924F925F926F923F
:103200007F928F929F92AF92BF92CF92DF92EF9276
:10321000FF920F931F93DF93CF93CDB7DEB728971D
:103220000FB6F894DEBF0FBECDBF1DC48091DE0582
:103230009091DF058330910509F448C184309105F0
:1032400034F4009781F0029709F0B0C116C18530BF
:10325000910509F47EC1853091050CF466C106978D
:1032600009F0A4C1DFC086EE95E060EC72E047E5AE
:1032700051E00E949C2AAC0186EE95E067E571E082
:103280000E94A12A9093E8058093E705892B61F1BC
:103290008AE190E00E94C904892B09F487C10E9449
:1032A000D8169093F2058093F105892B09F07EC121
:1032B0008091DE059091DF05892B09F077C186EEBC
:1032C00095E067E571E040E050E028EC30E00E94D6
:1032D000452B9093E8058093E70581E090E090937B
:1032E000F2058093F10562C18091550190915601DC
:1032F000039709F05BC12090C6053090C705409048
:10330000C8055090C90520E422162DE0320623E0BE
:10331000420620E0520638F400E1A02E07E2B02E6B
:10332000C12CD12C0CC0C201B10124E130E040E03D
:1033300050E00E944F32C901DA015C016D010E9428
:103340009A2C2091BE053091BF054091C005509147
:10335000C105621B730B840B950BA616B706C80636
:10336000D90608F023C10E949A2C7B018C01609041
:10337000C2057090C3058090C4059090C505E618FD
:10338000F70808091909C201B1012CE030E040E05A
:1033900050E00E944F322E153F054007510708F0BC
:1033A00005C18091BE059091BF05A091C005B09167
:1033B000C10586159705A805B90569F10E949A2CE3
:1033C0006093B6057093B7058093B8059093B905DF
:1033D00086EE95E00E94962AAA0CBB1CCC1CDD1C34
:1033E0008091C6059091C705A091C805B091C90507
:1033F0008A199B09AC09BD0980934D0190934E0138
:10340000A0934F01B093500185E090E09093DF05C9
:103410008093DE05CBC0A2E0B0E0B0935601A0934C
:103420005501C4C00E949A2C6093BA057093BB05E5
:103430008093BC059093BD052091B6053091B705EA
:103440004091B8055091B905621B730B840B950B25
:10345000673971058105910508F4A8C081E090E005
:103460000E94EB099093E8058093E70581E090E0E6
:103470009093F2058093F10595C00E949A2C2091BB
:10348000B6053091B7054091B8055091B905621B5A
:10349000730B840B950B6A3F71058105910508F448
:1034A00085C081E090E00E94EB099093E80580934D
:1034B000E70581E090E09093F2058093F105E3E069
:1034C000F0E0F093DF05E093DE0570C00E949A2CD7
:1034D0002091B6053091B7054091B8055091B905D6
:1034E000621B730B840B950B645F714080409040AE
:1034F00008F45CC086EE95E00E94962A8091550102
:1035000090915601892B31F082E090E09093560122
:1035100080935501A4E0B0E0B093DF05A093DE05F1
:1035200080E090E00E948E0F41C00E94DF2B20912E
:10353000B2053091B3054091B4055091B5052617F9
:1035400037074807590790F581E090E00E948E0FF9
:103550001BC00E949A2C2091B6053091B70540916E
:10356000B8055091B905621B730B840B950B209124
:103570004D0130914E0140914F0150915001621721
:1035800073078407950790F086EE95E00E94992ACC
:103590000E949A2C6093C2057093C3058093C40562
:1035A0009093C5051092DF051092DE050E949A2CBB
:1035B0002091510130915201409153015091540199
:1035C000621B730B840B950B6153754780409040D1
:1035D00030F18091DE059091DF05069701F180EAD8
:1035E00060E00E94EC0E1092A9051092A8050E94BE
:1035F0009A2C20E335E740E050E00E944F32CA01A8
:10360000B90120E335E740E050E00E9409326093C1
:103610005101709352018093530190935401809112
:10362000F1059091F205019709F046C10E949A2C8C
:103630002091BE053091BF054091C0055091C10554
:10364000621B730B840B950B615177428040904055
:1036500058F102ED15E00BC0F80180819181A28143
:10366000B38184839583A683B78304501040F5E02B
:10367000063C1F0789F71092F4051092F3050E948B
:103680009A2C2091BE053091BF054091C005509104
:10369000C105621B730B840B950BD80114966D93B7
:1036A0007D938D939C9317970E949A2C6093BE05EF
:1036B0007093BF058093C0059093C105209155017B
:1036C00030915601223031050CF4D9C06090CA0502
:1036D0007090CB058090CC059090CD05611471045D
:1036E0008104910409F4CBC02090CE053090CF0521
:1036F0004090D0055090D10521143104410451046B
:1037000009F4BDC08091D2059091D305A091D40554
:10371000B091D5058D839E83AF83B8870097A105AF
:10372000B10509F4ACC08091D6059091D705A09160
:10373000D805B091D90589839A83AB83BC83009760
:10374000A105B10509F49BC082017101E60CF71CCB
:10375000081D191D8D819E81AF81B885E80EF91E67
:103760000A1F1B1F89819A81AB81BC81E80EF91E5B
:103770000A1F1B1FB2E016950795F794E794BA95B8
:10378000D1F7E092C605F092C7050093C8051093E3
:10379000C905D801C701805C944DA140B040815457
:1037A0009840AC46B04008F061C0C801B70124E1C0
:1037B00030E040E050E00E944F32C901DA01570189
:1037C0006801A81AB90ACA0ADB0A6A147B048C04C5
:1037D0009D0408F43EC09C01AD012E0D3F1D401F0D
:1037E000511F261537054805590598F12A143B0441
:1037F0004C045D0470F1221533054405550548F16C
:103800008D819E81AF81B8858A159B05AC05BD056C
:1038100000F1281739074A075B07D8F089819A8198
:10382000AB81BC818A159B05AC05BD0590F02817BE
:1038300039074A075B0768F080915501909156015E
:103840000297E9F4A3E0B0E0B0935601A0935501CC
:1038500016C08091550190915601039781F4E2E0E2
:10386000F0E0F0935601E093550109C02330310593
:1038700031F482E090E0909356018093550140919D
:10388000E7055091E80586EE95E067E571E00E9456
:103890003A2BE7E5F1E080E090E002C0119201965A
:1038A000A2E0803C9A07D0F39093F4058093F3054F
:1038B0001092F2051092F1050E947508909356013E
:1038C0008093550182E00E94FB2D9093F405809334
:1038D000F3054091ED055091EE056091EF05709173
:1038E000F0050097D9F4411551056105710559F4AA
:1038F0000E949A2C6093ED057093EE058093EF057E
:103900009093F005A9C00E949A2C6093E9057093EA
:10391000EA058093EB059093EC059EC04115510597
:103920006105710509F459C08091E9059091EA0596
:10393000A091EB05B091EC050097A105B10509F444
:103940004CC08E5E9240A040B040841B950BA60BED
:10395000B70B835E9440A040B04008F03EC060E0EA
:1039600070E08091AC059091AD05892B11F461E078
:1039700070E07093AD056093AC0589E00E94A72DBF
:103980008091AC059091AD052091E4053091E5055D
:10399000019789F4232B21F48DE191E00E94FA072D
:1039A00087E090E09093DF058093DE0586EE95E05A
:1039B0000E94962A12C0232B21F484E191E00E94F8
:1039C000FA0781E090E00E948E0F86EE95E00E945B
:1039D000992A1092DF051092DE051092E9051092E7
:1039E000EA051092EB051092EC051092ED0510928D
:1039F000EE051092EF051092F0052EC06091A8051B
:103A00007091A905695E7B4F80EB97E041E050E043
:103A10000E94E531019749F48091A8059091A9058C
:103A200001969093A9058093A8058091A80590918F
:103A3000A905849731F480913A048F3711F40E94DC
:103A40000A068091A8059091A9058036910524F079
:103A50001092A9051092A80580EB97E00E945F2FB5
:103A6000181619065CF28091E0059091E105892B0A
:103A700009F0DCCB28960FB6F894DEBF0FBECDBFA1
:103A8000CF91DF911F910F91FF90EF90DF90CF903A
:103A9000BF90AF909F908F907F906F905F904F906E
:103AA0003F902F9008950F931F93CF93DF938C0136
:103AB000C0E0D0E0F801EC0FFD1F80EB97E06081E3
:103AC0004AE050E00E945131C330D10531F080EB23
:103AD00097E062E271E00E94B6312196C430D105D0
:103AE00049F7DF91CF911F910F9108954F925F9207
:103AF0006F927F928F929F92AF92BF92CF92DF92FE
:103B0000EF92FF920F931F93DF93CF9300D0CDB727
:103B1000DEB782E060E00E94682D89E061E00E94EB
:103B2000682D82E00E94FB2D019711F40E949C0FEA
:103B300085E10E94462D10E0662477246AE070E05B
:103B400080E090E00E94A82C85E10E94462D680E3E
:103B5000791E1F5F153091F740904301509044014A
:103B600081EE681685E0780634F081E090E090936D
:103B7000E5058093E40580EB97E040E855E260E0DE
:103B800070E00E94D82E80EB97E00E9409308823D5
:103B9000D1F38AE291E00E94FA0786EE95E00E9456
:103BA0008E2B86EE95E00E94992A86EE95E068E2DB
:103BB00071E00E948A2B80912E01882309F065C054
:103BC00080912F01882309F060C080913001882303
:103BD00009F05BC080913101882309F056C08091C3
:103BE000E4059091E505892B21F485EC91E00E9494
:103BF000FA0700D086E391E0EDB7FEB792838183A8
:103C000086EE95E067E571E040EC52E028E231E0B5
:103C100000E510E0BEE2EB2EB1E0FB2EAEE3CA2ED3
:103C2000A1E0DA2EF2E3AF2EF1E0BF2EEAE38E2E12
:103C3000E1E09E2E0E94A62A0F900F902091E405AD
:103C40003091E505882339F0232BF9F48FEB91E0CF
:103C50000E94FA071AC0232B21F489EA91E00E94FE
:103C6000FA0730EC30932E0128EA20932F0191E0DF
:103C70009093300189E18093310130933201209398
:103C8000330190933401909335012091420186EEE7
:103C900095E068E271E04EE251E030E00E944B2B8B
:103CA00086EE95E062E371E00E94362B8BE991E0AD
:103CB0000E94FA078091E2079091E307009711F4C0
:103CC00086EE97E0BE016F5F7F4F681B790B80EB3C
:103CD00097E04AE050E00E94A3318DE891E00E9415
:103CE000FA070E94CE07AB01BC0180EB97E02AE007
:103CF00030E00E94633182E891E00E94FA07B3014C
:103D0000882777FD8095982F920140E050E00E942F
:103D1000093220E034E140E050E00E944F3280EB75
:103D200097E0BA01A9012AE030E00E9442318DE714
:103D300091E00E94FA078091E4059091E505892BB6
:103D4000E1F480E791E00E94FA078EE291E00E94A0
:103D5000531D84E691E00E94FA078EE391E00E94F1
:103D6000531D88E591E00E94FA0782E391E00E94EA
:103D7000531D80EB97E00E94A2301092AB05109289
:103D8000AA051092A9051092A8051092D6051092C6
:103D9000D7051092D8051092D9051092D20510922D
:103DA000D3051092D4051092D5051092CE0510922D
:103DB000CF051092D0051092D1051092CA0510922D
:103DC000CB051092CC051092CD050E949A2C6093E1
:103DD000C2057093C3058093C4059093C505609395
:103DE000BE057093BF058093C0059093C10581E027
:103DF00090E00E948E0F1092DF051092DE0581E0A8
:103E000090E09093E1058093E0050F900F90CF91A3
:103E1000DF911F910F91FF90EF90DF90CF90BF90B7
:103E2000AF909F908F907F906F905F904F9008958C
:103E3000EF92FF920F931F938091D906853011F571
:103E4000E090DE06F090DF060091E0061091E106BA
:103E50008091DA069091DB06A091DC06B091DD0638
:103E6000E80EF91E0A1F1B1F0E949A2CAA2797FD15
:103E7000A095BA2F8E159F05A007B10718F086E010
:103E80008093D9068091D9061F910F91FF90EF90F2
:103E9000089585E08093D9060E949A2CAA2797FD61
:103EA000A095BA2F8093DA069093DB06A093DC06E8
:103EB000B093DD060E94C62282E00895FF920F9320
:103EC0001F93CF93DF938C01F62E1092E20610928F
:103ED000E3068091E4068F5F8093E40680E991E039
:103EE000D801FC011D923197E9F76091E40670E07A
:103EF000706E4091D4075091D507C80124E430E09A
:103F00000E941326D80116962091E5063091E60608
:103F1000C901FC0186E001900D928150E1F7C801D2
:103F20006FEF70E046E050E00E94F70282E8D801AF
:103F300051968C93519781E157968C938FEF9FEF19
:103F4000AFEFBFEFF801868F978FA0A3B1A383E4F3
:103F500085A312A284E483A3BA9681E0D8019A963D
:103F60008C93818386E0828313828091D306909123
:103F7000D406A091D506B091D60684839583A683F6
:103F8000B7838091D7069091D80691878087D80112
:103F9000DA961D921D921D921C92DD977C962091BF
:103FA000E5063091E606C901DC0186E00D9001923C
:103FB0008150E1F7D801AA5EBE4F93E6FD019193CF
:103FC00082E811968C93DF01119683E58183FD01D0
:103FD000319611969C93DF01119685E38183FD0153
:103FE000319691E011969C93DF011196F1829D012B
:103FF0002F5F3F4F8DE311968C93F901319687E047
:10400000D90111968C939183EF0122964091E50698
:104010005091E60620E030E0FE01E20FF31FDA01E6
:10402000A20FB31F8C9180832F5F3F4F2630310545
:1040300099F78CE08E838AE08F83289620E030E029
:10404000FE01E20FF31FD901A958BA4F8C9180836A
:104050002F5F3F4F2A30310599F72A96D093E80613
:10406000C093E7062A97B3E0FB1609F042C082E34B
:104070008A8794E09B87E091D407F091D5078081EF
:104080008C87E091D407F091D50781818D87E091ED
:10409000D407F091D50782818E87E091D407F09103
:1040A000D50783818F8786E3888B998B6296D0931F
:1040B000E806C093E7066297E091D607F091D7072C
:1040C00080818A8BE091D607F091D70781818B8B15
:1040D000E091D607F091D70782818C8BE091D607CB
:1040E000F091D70783818D8B6696D093E806C093B5
:1040F000E706A091E706B091E806FD0187E381930A
:1041000093E011969C93DF01119681E081839D01DC
:104110002F5F3F4F11969C93F901319686E0D901AC
:1041200011968C938FEF81833296F093E806E0939B
:10413000E706E01BF10BBA97C801BF010E94712787
:10414000DF91CF911F910F91FF90089563E070E090
:104150000E945E1F83E08093D9060895DF92EF925C
:10416000FF920F931F93CF93DF938C017B01E0911C
:10417000D407F091D507EC018AAD9BADACADBDADD8
:1041800080839183A283B383F801E65EFE4FE00E45
:10419000F11EDF011196D180ED01219680818630DC
:1041A000C1F0873030F4813051F0833009F057C0CE
:1041B0000BC0833399F0863309F051C042C0E091BF
:1041C000DA07F091DB0741C0E091D807F091D907F9
:1041D0003CC0E091D207F091D30737C011966C91A3
:1041E00070E080E090E0982F872F762F6627298156
:1041F000620F711D811D911D982F872F762F6627C5
:104200002A81620F711D811D911D982F872F762F96
:1042100066272B81620F711D811D911D982F872F9D
:10422000762F662728EE33E040E050E00E94093206
:104230006093DE067093DF068093E0069093E106BC
:104240000EC0E091D607F091D70711968D919D9100
:104250000D90BC91A02D80839183A283B383FE0136
:10426000ED0DF11DEE15FF0508F493CFC8010E9476
:10427000A62081E0DF91CF911F910F91FF90EF90E9
:10428000DF900895FC0166347105A0F183A18334A9
:1042900089F5DF019A9682A5823061F514962D91F9
:1042A0003D914D915C9117978091D3069091D406E2
:1042B000A091D506B091D606281739074A075B07A3
:1042C000C9F4E65EFE4F8081EA51F140853391F4F6
:1042D000E45EFE4F8081EC51F140823019F0853070
:1042E00049F404C0CF010E94AE200895CF010E947E
:1042F000491F089580E00895CF92DF92EF92FF92D8
:104300000F931F93CF93DF93EC017093E6066093B6
:10431000E5065093D5074093D4073093DB072093ED
:10432000DA071093D9070093D807F092D707E092E5
:10433000D607D092D307C092D20780E090E00E94C7
:10434000462D0E94D5020E94D002AA2797FDA09573
:10435000BA2F8F5D9C4BAA49BF4F8093D306909391
:10436000D406A093D506B093D6061092D806109224
:10437000D70680E090E0E091D407F091D507E80FF0
:10438000F91F1082E091DA07F091DB07E80FF91FBF
:104390001082E091D807F091D907E80FF91F108239
:1043A000E091D607F091D707E80FF91F1082E0914E
:1043B000D207F091D307E80FF91F108201968430DD
:1043C0009105C9F6E091E506F091E60685818295B2
:1043D0008F708F5B80937F0585818F708F5B80935B
:1043E00080050E94CF22CE0161E070E00E945E1F36
:1043F00081E08093D906DF91CF911F910F91FF90BB
:10440000EF90DF90CF9008958AE061E00E94682DE0
:104410008AE061E00E94A72D8BE061E00E94682D98
:104420008DE061E00E94682D8CE060E00E94682DC4
:104430008BE061E00E94A72D8BE060E00E94A72D39
:104440008DE060E00E94A72D81E58CBD8DB5816077
:104450008DBD08950F931F93CF93DF938C01EB01D4
:10446000F8948091820560E00E94A72D8AE78EBDB6
:104470000DB407FEFDCF08C088818EBD0DB407FEC8
:10448000FDCF21960150104001151105A9F780912B
:10449000820561E00E94A72D7894DF91CF911F9152
:1044A0000F9108950F931F93CF93DF93EC018B012E
:1044B000F8948091820560E00E94A72D8AE38EBD6A
:1044C0000DB407FEFDCF09C01EBC0DB407FEFDCF25
:1044D0008EB5F80181938F0121972097A9F78091DC
:1044E000820561E00E94A72D7894DF91CF911F9102
:1044F0000F910895FF920F931F93082F162FF42EFC
:10450000F8948091820560E00E94A72D1F71102B06
:104510001EBD0DB407FEFDCFFEBC0DB407FEFDCFE2
:104520008091820561E00E94A72D78941F910F91E0
:10453000FF9008951F93182F282F30E020763070B9
:104540008091E90690E02817390781F080EA6FE151
:1045500043E00E947A22412F40764093E90642953B
:104560004695477080E86FE10E947A221F91089576
:104570000F931F93182F062F0E949A2280E4612F19
:10458000402F0E947A221F910F9108956091EC06AE
:104590006E7F6093EC0688E30E94B82208956091D4
:1045A000EC0661606093EC0688E30E94B8220895EF
:1045B000682F677085E70E94B82208950F931F93B4
:1045C000182F072F0E94B822812F8F5F602F0E9423
:1045D000B8221F910F9108950F931F93182F062F44
:1045E000F8948091820560E00E94A72D802F8F7142
:1045F000812B8EBD0DB407FEFDCF1EBC0DB407FE92
:10460000FDCF07FF04C01EBC0DB407FEFDCF1EB5D5
:104610008091820561E00E94A72D7894812F1F91DF
:104620000F9108951F93182F0E949A2280E0612F06
:104630000E94EC221F910895AF92BF92CF92DF9219
:10464000EF92FF920F931F93DF93CF9300D0CDB7DC
:10465000DEB76C015B0189E30E941223882319F401
:1046600000E010E051C06091EA067091EB0680E036
:104670000E94DE2282E090E08E010F5F1F4FB801A2
:104680000E94522289819A819093EB068093EA06D8
:1046900082E090E0B8010E945222E980FA8082E034
:1046A00090E0B8010E945222898187FD03C000E09A
:1046B00010E00DC0C701049786010150104080171B
:1046C000910708F48C01C801B5010E945222609143
:1046D000EA067091EB068CE00E94DE226091EA0609
:1046E0007091EB066150704089E16F3F780720F0D0
:1046F0008CE06EEF79E101C08CE00E94DE2280E860
:104700006EE140E40E947A22C8010F900F90CF9191
:10471000DF911F910F91FF90EF90DF90CF90BF90AE
:10472000AF90089580EA6EE140E20E947A228DE126
:104730000E9412238823D9F380E86FE144E00E94AD
:104740007A22089580EA6FE144E00E947A228DE1A6
:104750000E94122382FDFBCF8FE10E94122383FD72
:10476000FBCF80E86EE148E00E947A2280E86EE1AB
:1047700040E20E947A2208950F931F93CF93DF9314
:10478000EC018B010FC08CE10E94122381FF0AC053
:1047900080E86FE140E80E947A2280EA6FE140E819
:1047A0000E947A2280E06FE10E94EC2283FDEBCF31
:1047B00082E06FEF79E10E94DE22BE016150764E09
:1047C00086E00E94DE228AE760E040E00E947A22D2
:1047D000CE01B8010E942A2280E86FE148E00E94E1
:1047E0007A22DF91CF911F910F9108950F931F931C
:1047F000982F162F072F84ED692F0E94B82286ED7F
:10480000612F0E94B82287ED602F0E94B82204C059
:104810008FE090E00E94012D8AEE0E94122380FD1D
:10482000F7CF1F910F9108950F931F938C01862F3F
:104830006093820561E00E94682D8091820561E0AD
:104840000E94A72D78948FEF60E04FEF0E947A22AC
:1048500062E370E080E090E00E94A82C1092EB06EA
:104860001092EA0688E060E070E00E94DE228CE0B0
:1048700060E070E00E94DE228AE06EEF79E10E9443
:10488000DE2284E06FEF79E10E94DE2286E06FEFA6
:104890007FE10E94DE2281EB8093EC0688E361EBEE
:1048A0000E94B82288E26FE370E30E94DE2280E378
:1048B00069EF77EF0E94DE2280EC6DE00E94B82263
:1048C00081EC60E00E94B82280E862EC42E30E9442
:1048D0007A2286EC62E17CE00E94DE2284EC62E1D6
:1048E0000E94B8228AEC6CED75E00E94DE2284EE14
:1048F000F80160810E94B82285EEF80161810E9472
:10490000B82282EEF80162810E94B82283EEF8019B
:1049100063810E94B82280EEF80164810E94B8226F
:1049200081EEF80165810E94B82280E160E071E0CB
:104930000E94F6238FE10E949A2280E86BE140EC0E
:104940000E947A2280E86FE144E00E947A221F915F
:104950000F910895682F84ED0E94B82282ED61E0E6
:104960000E94B8228FE090E00E94012D8AEE0E9402
:10497000122380FDFBCF82ED60E00E94B82289ED1A
:104980000E94122390E0089581E10E94AA2420E071
:10499000892B09F021E0822F0895CF92DF92EF92C8
:1049A000FF920F931F93CF93DF936C01413081F4FB
:1049B000685070407B0100E010E0685F7F4F21E1AC
:1049C00030E040E050E0E20EF31E041F151F15C05A
:1049D000423021F0EE24FF2487010FC06850704060
:1049E0007B0100E010E0685F7F4F86E090E0A0E090
:1049F000B0E0E80EF91E0A1F1B1FF601EB0116C0FE
:104A0000808190E0A0E0B0E0BA2FA92F982F8827EE
:104A1000218130E040E050E0822B932BA42BB52B7A
:104A2000E80EF91E0A1F1B1F32962297C230D105CD
:104A300038F7FB01EE7FEC0DFD1D60FF15C0808196
:104A400090E0A0E0B0E0BA2FA92F982F882708C0E7
:104A50002FEF3FEF40E050E0E222F3220423152342
:104A6000E80EF91E0A1F1B1FC801AA27BB270097C3
:104A7000A105B10569F7970120953095C901DF912E
:104A8000CF911F910F91FF90EF90DF90CF900895FD
:104A9000CF93DF93EC015093F3064093870520E01A
:104AA00030E0F901E65FF84FDB01A20FB31F8C91F4
:104AB00080832F5F3F4F2430310599F720E030E0AD
:104AC000F901E452F84FDE01A20FB31F8C918083ED
:104AD0002F5F3F4F2630310599F7DF91CF91089531
:104AE000FC0169327105B0F08485883099F48585C0
:104AF000863081F4DF019696EAE0F7E09C918081B0
:104B0000981741F41196319687E0EE30F807B1F727
:104B100081E0089580E00895FC016A327105D0F0CB
:104B200084858830B9F485858823A1F48685853409
:104B300089F4DF01EAE0F7E05E969C915E97808160
:104B4000981741F41196319687E0EE30F807A1F7F7
:104B500081E0089580E008950F931F938C01FC017C
:104B6000108E118E80E4848B158A868BC8010E9678
:104B700064E170E040E00E94CD24F801908F818FC5
:104B80001F910F910895AC01FC01AAE0B7E0828D5E
:104B9000868F8D91828F319687E0AE30B807B9F756
:104BA000CA010E94AC250895FC01B99694E0808169
:104BB000680F711D84816483442311F0808301C0D8
:104BC000108291503197992319F0672F7727EFCFF3
:104BD00008950F931F938C01FC0194A182A184A3DB
:104BE00092A395A183A185A393A3C8010E94D42574
:104BF000F80112AA13AA80E586A71F910F910895C4
:104C00006A5C7F4FDC01A60FB71F6653704003C07C
:104C10008D936F5F7F4FFA014F5F5F4F84918823C1
:104C2000B9F7CB010895FF920F931F93CF93DF93B2
:104C3000EC01F62E072FBA01122F932FAE019E0121
:104C4000A0E0B0E0FD01E050F94F8081F9018083E0
:104C5000FD01E452F84F8081F901868311962F5FA0
:104C60003F4FA630B10571F788E08C871D86DE01C5
:104C7000EFE3F3E084911E968C931E973196119684
:104C800083E0E834F807B1F7188A81E18F8BA0E060
:104C9000B0E0FB01EA0FFB1F8081FA01868FFD0166
:104CA000E65FF84F8081FA01828F11964F5F5F4F68
:104CB000A430B10571F79CA31DA30AA3FBA21EA2F9
:104CC00018A619A6DF91CF911F910F91FF9008951B
:104CD000AC0181E08093830520E030E0F901E450ED
:104CE000F94FDA01A20FB31F8C9180832F5F3F4FE2
:104CF0002430310599F70895CF93DF93EB01BA0182
:104D0000DA010D900020E9F71197A41BB50BE69688
:104D1000AC014C0F5D1FE6979D0108C0FB0181911E
:104D2000BF01FA018193AF012150304021153105B7
:104D3000A9F79E012A0F3B1FC901DF91CF9108956A
:104D4000FF920F931F93CF93DF93EC01F62E142F56
:104D5000022FAC01DC0120E030E0F901E050F94F16
:104D600080818C93F901E452F84F808116968C93E0
:104D700016972F5F3F4F11962630310571F788E067
:104D80008C871D86DE01EFE3F3E084911E968C9301
:104D90001E973196119683E0E834F807B1F78CE25C
:104DA000898B86E08F8B20E030E0F901EA5FF84FD5
:104DB0008081FA01868FF901E65FF84F8081FA0160
:104DC000828F2F5F3F4F4F5F5F4F2430310569F770
:104DD000CE010E94AC251CA30DA38BE08AA3FBA2ED
:104DE000FE01B69680E011928F5F8830E1F78091E6
:104DF000880588A78D5F8093880580E68EA782E06E
:104E00008FA794E098AB19AA1AAA1BAA1CAA1DAADC
:104E10008EAB9FAB88AF86E289AFCE014A9660E247
:104E200070E042E00E94CD249AAB8BAB8AE390E025
:104E3000BE010E94BC23DF91CF911F910F91FF9083
:104E40000895CF93DF93EC01AC012CED37E0FC012A
:104E5000D9019FEF90838D918683319687E0A23EA2
:104E6000B807C1F788E08C8786E08D87DE01E7E32D
:104E7000F3E084911E968C931E973196119683E0F1
:104E8000EF33F807B1F7F90181919F01FA01868BA1
:104E900010A24F5F5F4FF7E0223E3F07A1F7DE0110
:104EA0005C9620E030E0FB01E20FF31F80811A9650
:104EB0008C931A97F901E65FF84F80818D932F5FED
:104EC0003F4F2430310579F78091830588608093C6
:104ED00083058AE290E0BE010E94BC23DF91CF915E
:104EE0000895DF92EF92FF920F931F938C017B0145
:104EF0008CE190E0E80EF91EF801F08A84EE9FEF55
:104F0000E80EF91EDE2C9CE1D90ED18AC8010E9460
:104F1000AC25E8E0F0E0EE0EFF1EF801F6A2FCEE94
:104F2000DF0EF801D7A288E090E0E80EF91EC80174
:104F30004A96B70141E00E94CD24F80190A781A7CD
:104F4000C7014A96B8010E94BC231F910F91FF90A0
:104F5000EF90DF900895EF92FF920F931F938C01D3
:104F60007B01CB018896F801908B818BC8010E9450
:104F7000AC25F80112AA13AA8CE190E0E80EF91E04
:104F8000C8014A96B70142E00E94CD24F80192ABD5
:104F900083ABC7014A96B8010E94BC231F910F91B1
:104FA000FF90EF900895CF93DF93EC01FC01ACEDFF
:104FB000B7E0868180838D918683319687E0A23E1B
:104FC000B807B9F7842F80618FA7443029F06115A5
:104FD000710511F461E070E0CE0141E00E94E92525
:104FE000188A88E2898BCE010E94C32584E088ABB1
:104FF00019AACE014A966CE170E042E00E94CD24ED
:105000009AAB8BAB86E390E0BE010E94BC23DF919C
:10501000CF910895EF92FF920F931F938C017B0124
:105020006091F4067091F50640E00E94D32789E173
:10503000F80187A7C801B7010E94AB271F910F9104
:10504000FF90EF900895CF93DF93EC01FC01ACED5E
:10505000B7E0868180838D918683319687E0A23E7A
:10506000B807B9F7188A8CE2898BCE010E94C32554
:1050700082E18FA7CE0161E070E040E00E94E92567
:105080001EA21FA28091880588A719A68D5F809314
:10509000880582E08EAB84E08FAB95E098AF19AEC7
:1050A00080E68EA798AB88E789ABCE014A9660E28E
:1050B00070E042E00E94CD249AAB8BAB8AE390E093
:1050C000BE010E94BC23DF91CF9108950F931F93DF
:1050D000CF93DF93EC018B01FC01ACEDB7E086814F
:1050E00080838D918683319687E0A23EB807B9F719
:1050F000CE010E94C3251AA28CA1883F18F08DA171
:105100008F5F8DA38CA1885F8CA3C801BE010E9414
:10511000BC23DF91CF911F910F910895CF93DF931F
:10512000AC01EC012CED37E0FC01D90186818083D4
:105130008D918683319687E0A23EB807B9F7FA01D0
:10514000148A82E0858B8E8988A3F90181919F0161
:105150008E8B2196F7E0223E3F07A9F7FA017C9655
:10516000AAE0B7E0808182878D91819387E0AE309D
:10517000B807C1F78AE290E0BA010E94BC23DF9130
:10518000CF910895EF92FF920F931F93CF93DF93E8
:10519000EC017B016115710509F040C08091830528
:1051A00080FD04C08091830582FF0FC0809184053B
:1051B00090918505892B49F40E94C424882329F005
:1051C000CE016CEF76E00E942127809184059091BA
:1051D0008505019690938505809384058091ED0661
:1051E000813009F08FC18091830581FF8BC182E0FE
:1051F0008093ED06809186058F5F809386058F7181
:105200006091EE066295660F607E682BCE0140913C
:10521000EF062091F0060E94A02674C10E9470251E
:10522000882341F18D89813019F4CE010E948E28A6
:105230008091830583FF66C18D89823009F062C148
:10524000ECEFF6E0DE015C969C915C97808198170C
:1052500009F058C11196319687E0E030F80799F7C8
:10526000E0E0F7E08E898193219697E0E630F90738
:10527000C9F752C1CE01B7010E948C25882309F4D9
:1052800041C19F89913149F48AA18823C9F48BA136
:105290008533B1F46AE270E037C1913089F48AA1B4
:1052A000883071F4E091FA06F091FB06309719F01E
:1052B000CE014A960995CE01B7010E94662822C107
:1052C00086E3E816F10418F4963009F01BC19CA19E
:1052D0009B3009F0C9C0D093F206C093F106DE01FD
:1052E000E6E0F7E05A969C915A978081981709F06A
:1052F00009C11196319697E0EA30F90799F710C184
:10530000E091F606F091F706309709F4A3C08DA15D
:1053100082958695877063E040E050E020E030E0C1
:10532000099598C0988980E02989022F10E0082B00
:10533000192B8EA582958F70482F50E0CA01880FD7
:10534000991F880F991F081B190B0451104017FF54
:1053500002C000E010E0B8018091ED06823089F5CE
:1053600031FF20C034FF1EC0CE0160E070E040E09D
:105370000E94D32788E18FA7E091F806F091F90603
:10538000309719F460E070E006C08BA18295869595
:1053900087700995BC0183E08093ED06CE010E94E1
:1053A000AB27B0C081E08093ED068FA584FF03C0DA
:1053B00060E070E003C0B8016F5F7F4FCE0144E052
:1053C0008CC0843039F4E091F606F091F7063097FE
:1053D00089F432C0833099F584E08093ED06E09142
:1053E000F606F091F706309739F18EA582958F7009
:1053F000482F50E0440F551F440F551FC701089711
:105400004E5D5F4F8417950708F4AC01C801840F07
:10541000951FE816F90610F0980103C09701241BA8
:10542000350B8DA182958695877060E0099588235C
:1054300019F0CE01B8010BC0CE01B8014DC08530C6
:1054400009F460C030FF0AC06F5F7F4FCE0149E0B2
:105450000E94D32785E08093ED0654C00115110505
:1054600009F452C0CE0138C08091F306981709F0B4
:1054700049C09DA180918705981709F043C08FA569
:1054800081FF04C0CE010E9423283CC084FF3AC0A3
:10549000988980E02989422F50E0482B592B2EA56E
:1054A000822F82958F7090E0880F991F880F991F27
:1054B000481B590B4451504057FF02C040E050E098
:1054C0005093F5064093F406452B51F48FA580FFC9
:1054D00019C0CE0160E070E040E00E94D32712C006
:1054E0008EA582958F70682F70E0660F771F660F0C
:1054F000771F6E5D7F4F88EF9FEFE80EF91EE6166F
:10550000F70610F460E070E0CB01DF91CF911F91BE
:105510000F91FF90EF90089582E080938305F2CF82
:105520008FA5382F82FDECCEFDCE08950E94A223D8
:1055300008950E9492230895CB01BA010E941C2372
:105540000895CB01BA010E94C22808952F923F927C
:105550005F926F927F928F929F92AF92BF92CF9203
:10556000DF92EF92FF920F931F93DF93CF93CDB70C
:10557000DEB72A970FB6F894DEBF0FBECDBF3B0152
:105580005A8349833C832B83FE82ED82D886CF8267
:10559000BA86A98614010E949A2CAC01CB01DA01CB
:1055A0004C015D01C3016B817C814D815E812F8146
:1055B000388509851A857101CE8CDF8C0E947C218B
:1055C00088E0582E89819A81B3010E941C238C01A6
:1055D000C301B8010E94C228892BA1F7C301B801F9
:1055E0000E9442210E94181F853011F481E026C0DC
:1055F0000E949A2CA50194012059384E4F4F5F4FBD
:105600002617370748075907E8F60E949A2C5A943C
:10561000A1F0AC01CB01DA014C015D01C3016B814A
:105620007C814D815E812F81388509851A857101C4
:10563000CE8CDF8C0E947C21C5CF80E02A960FB6ED
:10564000F894DEBF0FBECDBFCF91DF911F910F91B8
:10565000FF90EF90DF90CF90BF90AF909F908F9092
:105660007F906F905F903F902F900895CB010E94A4
:1056700068260895CB01BA010E940A280895CB013B
:10568000BA01A9010E947C260895CB01BA01A901A3
:105690000E9400260895CB01BA01A9010E94482565
:1056A0000895CF93DF93CB01642F0E94142482E0EE
:1056B0000E94D8226AE070E080E090E00E94A82C6E
:1056C000C0E0D0E084E160E878E30E94F62364EF74
:1056D00071E080E090E00E94A82C84E160E979E329
:1056E0000E94F62364EF71E080E090E00E94A82C15
:1056F0002196C330D10531F784E166E774E30E9457
:10570000F62364E670E080E090E00E94A82CDF9130
:10571000CF9108954AE00E94512B08950E940422DF
:105720000895F999FECF72BD61BDF89A80B50895CC
:10573000F999FECF1FBA72BD61BD40BD0FB6F89496
:10574000FA9AF99A0FBE08958091190790911A0755
:1057500008956093890570938A0580938B059093D3
:105760008C050895609311077093120780931307B7
:10577000909314072091890530918A0540918B05FB
:1057800050918C05260F371F481F591F209315076E
:1057900030931607409317075093180782E090E064
:1057A00090931A07809319070E949A2C60931B0705
:1057B00070931C0780931D0790931E070895EF9226
:1057C000FF920F931F931CC02F5F3F4F4F4F5F4FB0
:1057D0002093110730931207409313075093140737
:1057E00088EE93E0A0E0B0E0E80EF91E0A1F1B1F50
:1057F000E0921B07F0921C0700931D0710931E07F1
:105800000E949A2CE0901B07F0901C0700911D0746
:1058100010911E076E197F09800B910B20911107C3
:10582000309112074091130750911407685E73403E
:105830008040904048F68091150790911607A091FE
:105840001707B0911807281739074A075B07E8F0D0
:10585000E0910F07F0911007309749F00995611515
:1058600071058105910519F00E94B22B0EC020E050
:1058700030E08091190790911A07892B11F021E0EF
:1058800030E030931A072093190760911107709147
:10589000120780911307909114071F910F91FF90A9
:1058A000EF9008951F920F920FB60F9211242F932D
:1058B0003F938F939F93AF93BF93809123079091D2
:1058C0002407A0912507B09126073091270701965C
:1058D000A11DB11D232F2D5F2D3720F02D570196CF
:1058E000A11DB11D209327078093230790932407C0
:1058F000A0932507B093260780911F07909120075A
:10590000A0912107B09122070196A11DB11D80939E
:105910001F0790932007A0932107B0932207BF9100
:10592000AF919F918F913F912F910F900FBE0F904C
:105930001F9018958FB7F894209123073091240772
:1059400040912507509126078FBFB901CA010895DC
:105950009B01AC017FB7F89480911F0790912007BD
:10596000A0912107B091220766B5A89B05C06F3FA3
:1059700019F00196A11DB11D7FBFBA2FA92F982F35
:105980008827860F911DA11DB11D62E0880F991F08
:10599000AA1FBB1F6A95D1F7BC012DC0FFB7F894B1
:1059A00080911F0790912007A0912107B0912207B5
:1059B000E6B5A89B05C0EF3F19F00196A11DB11DEA
:1059C000FFBFBA2FA92F982F88278E0F911DA11DD9
:1059D000B11DE2E0880F991FAA1FBB1FEA95D1F7FE
:1059E000861B970B885E9340C8F2215030404040A0
:1059F000504068517C4F211531054105510571F624
:105A00000895019739F0880F991F880F991F029701
:105A10000197F1F70895789484B5826084BD84B5C8
:105A2000816084BD85B5826085BD85B5816085BD99
:105A3000EEE6F0E0808181608083E1E8F0E01082B2
:105A4000808182608083808181608083E0E8F0E0F3
:105A5000808181608083E1EBF0E0808184608083DD
:105A6000E0EBF0E0808181608083EAE7F0E0808114
:105A70008460808380818260808380818160808374
:105A80008081806880831092C1000895982F8E30A5
:105A900008F09E50977080918D058295880F880F31
:105AA000807C892B80937C0080917A008064809335
:105AB0007A0080917A0086FDFCCF20917800409199
:105AC0007900942F80E030E0282B392BC90108950C
:105AD000CF93DF93482F50E0CA0183589B4FFC01BE
:105AE000349147595B4FFA018491882369F190E022
:105AF000880F991FFC01E55BFB4FA591B491FC0158
:105B0000EB5AFB4FC591D491662351F42FB7F8940B
:105B10008C91932F909589238C93888189230BC036
:105B2000623061F42FB7F8948C91932F909589236C
:105B30008C938881832B88832FBF06C09FB7F894EE
:105B40008C91832B8C939FBFDF91CF910895482F29
:105B500050E0CA018F569B4FFC012491CA01835823
:105B60009B4FFC01949147595B4FFA0134913323C9
:105B700009F440C0222351F1233071F0243028F47D
:105B80002130A1F0223011F514C02630B1F02730B9
:105B9000C1F02430D9F404C0809180008F7703C015
:105BA000809180008F7D8093800010C084B58F77B6
:105BB00002C084B58F7D84BD09C08091B0008F770D
:105BC00003C08091B0008F7D8093B000E32FF0E0A0
:105BD000EE0FFF1FEB5AFB4FA591B4912FB7F8942E
:105BE000662321F48C919095892302C08C91892B96
:105BF0008C932FBF0895682F70E0CB018F569B4F79
:105C0000FC012491CB0183589B4FFC0144916759BF
:105C10007B4FFB019491992319F420E030E03CC0C4
:105C2000222351F1233071F0243028F42130A1F0E7
:105C3000223011F514C02630B1F02730C1F02430E5
:105C4000D9F404C0809180008F7703C080918000D8
:105C50008F7D8093800010C084B58F7702C084B59B
:105C60008F7D84BD09C08091B0008F7703C0809183
:105C7000B0008F7D8093B000892F90E0880F991F2E
:105C8000815A9B4FFC01A591B4918C9120E030E0AA
:105C9000842311F021E030E0C901089508951F9296
:105CA0000F920FB60F9211242F933F934F938F9320
:105CB0009F93EF93FF938091C00082FD1DC04091A0
:105CC000C60020916807309169072F5F3F4F2F73FF
:105CD000307080916A0790916B072817390771F02F
:105CE000E0916807F0916907E85DF84F40833093D1
:105CF00069072093680702C08091C600FF91EF9169
:105D00009F918F914F913F912F910F900FBE0F90C8
:105D10001F901895E091BC07F091BD07E05CFF4F24
:105D20008191919120813181821B930B8F739070AF
:105D3000892B11F00E944E2E08951F920F920FB6DC
:105D40000F9211242F933F938F939F93EF93FF9381
:105D50002091AC073091AD078091AE079091AF07CD
:105D60002817390731F48091C1008F7D8093C100DD
:105D700014C0E091AE07F091AF07E459F84F2081CD
:105D80008091AE079091AF0701968F7390709093BA
:105D9000AF078093AE072093C600FF91EF919F91CC
:105DA0008F913F912F910F900FBE0F901F901895DC
:105DB000AF92BF92DF92EF92FF920F931F93CF9318
:105DC000DF93EC017A018B01DD24403081EE58072E
:105DD00080E0680780E0780711F0DD24D39491E03B
:105DE000A92EB12CEC89FD89DD2069F0C50108A040
:105DF00002C0880F991F0A94E2F7808360E079E07F
:105E00008DE390E005C0108260E874E88EE190E0D8
:105E1000A80197010E944F3221503040404050402D
:105E2000569547953795279580E12030380720F023
:105E3000DD2011F0DD24D6CFE889F9893083EA89A5
:105E4000FB89208319A2EE89FF89408121E030E09F
:105E5000C9010C8C02C0880F991F0A94E2F7482BE5
:105E60004083EE89FF894081C9010D8C02C0880FF3
:105E7000991F0A94E2F7482B4083EE89FF894081FD
:105E8000C9010E8C02C0880F991F0A94E2F7482BB3
:105E90004083EE89FF8980810F8C02C0220F331F5F
:105EA0000A94E2F7209528232083DF91CF911F9158
:105EB0000F91FF90EF90DF90BF90AF900895DC01BD
:105EC0001C96ED91FC911D97E05CFF4F2191319163
:105ED00080819181281B390B2F733070C90108957F
:105EE000DC011C96ED91FC911D97E05CFF4F208139
:105EF0003181E054F040DF01AE5BBF4F8D919C914A
:105F000011972817390719F42FEF3FEF07C08D912C
:105F10009C91E80FF91F8081282F30E0C901089576
:105F2000DC011C96ED91FC911D97E05CFF4F2081F8
:105F30003181E054F040DF01AE5BBF4F8D919C9109
:105F400011972817390719F42FEF3FEF10C08D91E3
:105F50009C911197E80FF91F20818D919C911197C9
:105F600001968F73907011969C938E9330E0C901C7
:105F70000895DC0191968C919197882339F054967D
:105F8000ED91FC915597808186FFF9CF91961C92F7
:105F90000895CF93DF93EC01EE85FF85E05CFF4F22
:105FA00020813181E054F0402F5F3F4F2F733070DC
:105FB000DF01AE5BBF4F8D919C9111972817390778
:105FC000D1F3E05CFF4F80819181E054F040E80F15
:105FD000F91F6083EE85FF85E05CFF4F31832083EE
:105FE000EE89FF89208181E090E00F8C02C0880F4C
:105FF000991F0A94E2F7282B208381E089A3EC897A
:10600000FD8980818064808381E090E0DF91CF9181
:10601000089581E008951092B3071092B20788EEB8
:1060200093E0A0E0B0E08093B4079093B507A0930D
:10603000B607B093B70782E995E09093B1078093D4
:10604000B00788E297E09093BD078093BC078CE689
:1060500097E09093BF078093BE0785EC90E0909304
:10606000C1078093C00784EC90E09093C3078093AE
:10607000C20780EC90E09093C5078093C40781EC41
:1060800090E09093C7078093C60782EC90E09093CE
:10609000C9078093C80786EC90E09093CB07809364
:1060A000CA0784E08093CC0783E08093CD0787E024
:1060B0008093CE0785E08093CF0781E08093D0075F
:1060C0000895CF93DF930E940B2D0E94761DCAE89E
:1060D000DEE20E94FB182097E1F30E948A2EF9CF9E
:1060E000CF92DF92EF92FF920F931F93CF93DF93A4
:1060F0007C016B018A01C0E0D0E00FC0D6016D9138
:106100006D01D701ED91FC910190F081E02DC70167
:106110000995C80FD91F015010400115110571F7DD
:10612000CE01DF91CF911F910F91FF90EF90DF9003
:10613000CF900895DC01ED91FC910190F081E02D6C
:1061400009950895EF92FF920F931F938C01DC0144
:10615000ED91FC910190F081E02D6DE009957C01BD
:10616000D801ED91FC910190F081E02DC8016AE029
:1061700009959C012E0D3F1DC9011F910F91FF90A4
:10618000EF900895CF93DF93EC016115710519F439
:1061900020E030E00FC0DB010D900020E9F71197FF
:1061A000A61BB70BE881F9810280F381E02DAD01D8
:1061B00009959C01C901DF91CF9108954F925F929B
:1061C0007F928F929F92AF92BF92CF92DF92EF9287
:1061D000FF920F931F93DF93CF93CDB7DEB7A197B5
:1061E0000FB6F894DEBF0FBECDBF2C01742ECB01CD
:1061F000223008F42AE019A231E2C32ED12CCC0EB1
:10620000DD1E822E9924AA24BB24672D752FA5019B
:1062100094010E944F3279018A01C801B701A5019A
:1062200094010E940932472D461B0894C108D108E9
:106230004A3014F4405D01C0495CF6014083E1142A
:10624000F1040105110521F07E2C5F2DC801DDCF81
:10625000C201B6010E94C230A1960FB6F894DEBF0B
:106260000FBECDBFCF91DF911F910F91FF90EF90A7
:10627000DF90CF90BF90AF909F908F907F905F9076
:106280004F900895DC012115310541F4ED91FC9109
:106290000190F081E02D642F099508950E94DE3071
:1062A0000895EF92FF920F931F939A01E62EFF2419
:1062B00000E010E0B801A7010E9442311F910F9148
:1062C000FF90EF900895CF92DF92EF92FF920F939D
:1062D0001F93CF93DF93EC016A017B0121153105F8
:1062E00041F4E881F9810190F081E02D642F099556
:1062F0001FC02A303105D1F477FF17C0E881F9813A
:106300000190F081E02D6DE209958C01442755271D
:10631000BA014C195D096E097F09CE012AE00E947D
:10632000DE309801280F391F04C02AE00E94DE30B9
:106330009C01C901DF91CF911F910F91FF90EF90C8
:10634000DF90CF900895EF92FF920F931F937B0100
:106350009A010027F7FC0095102FB801A7010E94B1
:1063600063311F910F91FF90EF9008950E94C2300A
:106370000895CF93DF93EC010E949A2C6887798768
:106380008A879B87E881F9810680F781E02DCE011D
:1063900009959C0197FF15C00E949A2C2885398584
:1063A0004A855B85621B730B840B950B2C813D81A9
:1063B0004E815F81621773078407950718F32FEFEB
:1063C0003FEFC901DF91CF910895CF92DF92EF9215
:1063D000FF920F931F93CF93DF936C018B017A0190
:1063E000C0E0D0E009C0C6010E94B93197FD07C0E6
:1063F000F80181938F012196CE15DF05A0F3CE0120
:10640000DF91CF911F910F91FF90EF90DF90CF9090
:106410000895629FD001739FF001829FE00DF11DEE
:10642000649FE00DF11D929FF00D839FF00D749F0E
:10643000F00D659FF00D9927729FB00DE11DF91FBA
:10644000639FB00DE11DF91FBD01CF011124089517
:10645000AA1BBB1B51E107C0AA1FBB1FA617B7078A
:1064600010F0A61BB70B881F991F5A95A9F78095A6
:106470009095BC01CD01089597FB092E07260AD0FF
:1064800077FD04D0E5DF06D000201AF47095619501
:106490007F4F0895F6F7909581959F4F0895A1E25B
:1064A0001A2EAA1BBB1BFD010DC0AA1FBB1FEE1F8E
:1064B000FF1FA217B307E407F50720F0A21BB30BD9
:1064C000E40BF50B661F771F881F991F1A9469F755
:1064D00060957095809590959B01AC01BD01CF01B1
:1064E000089597FB092E05260ED057FD04D0D7DF5F
:1064F0000AD0001C38F450954095309521953F4FB7
:106500004F4F5F4F0895F6F7909580957095619580
:106510007F4F8F4F9F4F0895EE0FFF1F0590F4910F
:10652000E02D09942F923F924F925F926F927F924B
:106530008F929F92AF92BF92CF92DF92EF92FF9293
:106540000F931F93CF93DF93CDB7DEB7CA1BDB0B3F
:106550000FB6F894DEBF0FBECDBF09942A883988E4
:1065600048885F846E847D848C849B84AA84B984EB
:10657000C884DF80EE80FD800C811B81AA81B981F7
:10658000CE0FD11D0FB6F894DEBF0FBECDBFED010B
:066590000895F894FFCF0E
:106596003F50313D002650323D002650333D002607
:1065A60050343D002650323D310047455420002FDF
:1065B60020002E0001000000545556212223C0A8B9
:1065C6000119C0A80101C0A80101C0A80101FFFF6F
:1065D600FF00501A4F9033C83240003A00204E0058
:1065E600001027000002000000000000000000006C
:1065F6000000000000000000000000000000000095
:106606000000000000000000000000000000000084
:106616000000000000000000000000000000000074
:106626000000000000000000000000000000000064
:106A06000000000000000041726475696E6F2D3051
:106A160030000A01010001500A2C010000010000AB
:0E6A26000000C92F70305F2F902F702FB92FF6
:00000001FF
